:100000002500A3046400FF0C2B002C001A0A270211
:1000100043070E0A280243060008E800E700140C14
:100020002900150AE902110A070A0E0C2A00EA0241
:10003000170A120A110C2D00210C2E00220C2F0081
:10004000120C3000080C2B000600A30466062A0AD6
:10005000A304490AA4040D022600190C2700680015
:10006000A30407090E022600190C27006800A30448
:1000700007090F022600190C27006800A3040709CE
:1000800010022600190C27006800A3040709A30426
:10009000250A0D022600190C27006800A304070991
:1000A00010022600190C27006800A30407090F029C
:1000B0002600190C27006800A30407090E02260079
:1000C000190C27006800A3040709A304250AA30448
:1000D000680A0000000000000000000000000000AE
:1000E0000000000000000000000000000000000010
:1000F0000000000000000000000000000000000000
:1001000000000000000000000000000000000000EF
:1001100000000000000000000000000000000000DF
:1007F0000000000000000000000000000000FE0CEF
:021FFE000A00D7
:00000001FF
